:020000040800F2
:10000000F005002049020008D5310008FF2E000845
:10001000D1310008C7140008253A0008000000008C
:10002000000000000000000000000000B1330008E4
:10003000E114000800000000D7310008B3330008C5
:100040006D0200086D0200086D0200086D020008D4
:100050006D0200086D0200086D0200086D020008C4
:100060006D0200086D0200086D0200086D020008B4
:100070006D0200086D0200086D0200086D020008A4
:100080006D0200086D0200086D0200086D02000894
:100090006D0200086D0200086D0200086D02000884
:1000A0006D0200086D0200086D0200086D02000874
:1000B0006D0200086D0200086D0200086D02000864
:1000C0006D0200086D0200086D0200086D02000854
:1000D0006D020008D53900086D0200086D020008A5
:1000E0006D0200086D0200086D0200086D02000834
:1000F0006D0200086D0200086D0200086D02000824
:100100006D0200086D0200086D0200086D02000813
:100110006D0200086D0200086D0200086D02000803
:100120006D0200086D0200086D0200086D020008F3
:100130006D0200086D0200086D0200086D020008E3
:100140006D0200086D0200086D0200086D020008D3
:100150006D0200086D0200086D0200086D020008C3
:100160006D0200086D0200086D0200086D020008B3
:100170006D0200086D0200086D020008000000001A
:100180006D0200086D02000800F002F800F04CF863
:100190000AA090E8000C82448344AAF10107DA45E2
:1001A00001D100F041F8AFF2090EBAE80F0013F0E8
:1001B000010F18BFFB1A43F001031847FC4700006A
:1001C0001C480000103A24BF78C878C1FAD85207FA
:1001D00024BF30C830C144BF04680C6070470000C1
:1001E0000023002400250026103A28BF78C1FBD840
:1001F000520728BF30C148BF0B607047662904F022
:100200008283642900F0FE80002070471FB504F04F
:1002100070FB00F013FC04000020002103F0FCFD43
:10022000E0601FBD10B510BD00F024FD1146FFF7C2
:10023000EDFF03F0ABFC00F042FD03B4FFF7F2FF6B
:1002400003BC03F062FC00000C48016841F470013B
:1002500001600B4880470B480047FEE7FEE7FEE7DA
:10026000FEE7FEE7FEE7FEE7FEE7FEE7FEE700004B
:1002700005480649044A064B7047000088ED00E037
:10028000BD33000889010008F0010020F0050020BE
:10029000F0010020704753EA020C00F069802DE95C
:1002A000F04B4FF00006002B1FBFB3FA83F503FAA3
:1002B00005F424FA05F65E4012BF1643B2FA82F541
:1002C00002FA05F4C5F120051EBF22FA05FC44EA36
:1002D0000C04203556EA044C4FEA144418BF641C41
:1002E0004FF000084FF00009904271EB030C39D336
:1002F000002919BFB1FA81F701FA07F6B0FA80F7C1
:1003000000FA07F6C7F120071EBF20FA07FC46EAED
:100310000C062037B6FBF4FCA7EB0507103F07F0EF
:100320001F0BCBF120060CFA0BFB2CFA06F644BF90
:10033000B3460026202FA4BF5E464FF0000B5BEAB9
:10034000060C08BF4FF0010B19EB0B09ABFB027C4D
:1003500048EB0608C01B06FB02CC0BFB03CC71EB81
:100360000C01C1E70B46024641464846BDE8F08B0A
:1003700013B54FF000004FF00001AFF30080BDE86F
:100380001C4070470FB4044910B503AA029800F04E
:1003900043FB10BC5DF814FB040000202DE9F04184
:1003A0000E460446002020622046E168884730B3AC
:1003B000252805D0D4E901219047206A401CF2E7A6
:1003C000E168204600278847050018D0A5F14100C4
:1003D000192802D820354FF40067324629462046B6
:1003E0002760FFF70BFF40B1012804D0F61D26F06F
:1003F00007060836D8E7361DD6E72846DAE7206A2A
:10040000BDE8F0812DE9F041064600241068752909
:10041000314616A510D0AFF30080002802DA404222
:1004200013A507E031688A0701D512A502E0490744
:1004300004D511A5012401E0AFF3008000210A22B8
:1004400006F1240709E0B0FBF2FCB0FBF2F302FB7B
:100450001C00303078541846491C0028F3D123463C
:100460002A463046BDE8F04100F070B800000000B8
:100470002D0000002B0000002000000010B5203AE5
:10048000C0F00B80B1E81850203AA0E81850B1E84D
:100490001850A0E81850BFF4F5AF5FEA027C24BF03
:1004A000B1E81850A0E8185044BF18C918C0BDE8FA
:1004B00010405FEA827C24BF51F8043B40F8043BC3
:1004C00008BF7047D20728BF31F8023B48BF11F878
:1004D000012B28BF20F8023B48BF00F8012B7047D2
:1004E0004FF0000200B5134694469646203922BFCD
:1004F000A0E80C50A0E80C50B1F12001BFF4F7AF18
:10050000090728BFA0E80C5048BF0CC05DF804EBF9
:10051000890028BF40F8042B08BF704748BF20F867
:10052000022B11F0804F18BF00F8012B7047704765
:1005300070477047704710B500F084FA006810BD2E
:1005400010B5044600F07EFA046010BD2DE9F047B6
:100550000D4699469246044600F124080168880633
:1005600004D5E06921F01001216000E00120A842DB
:1005700001DD471B00E00027A1697A1902EB0900A1
:10058000081AA0612078C00602D42046AFF300808C
:10059000002608E0D4E901211AF806009047206AF5
:1005A000401C761C20624E45F4DB2078C0060AD53C
:1005B0002046AFF3008006E0D4E9012130209047C7
:1005C000206A401C2062381EA7F10107F4DC07E016
:1005D000D4E9012118F805009047206A401C2062E8
:1005E000281EA5F10105F3DC2046AFF3008020783A
:1005F000000602D50220BDE8F0870120FBE7704726
:100600002DE9FF4F0C461E464FF0FF378BB0D2E965
:100610000001DDF860800A908A46C1F30A5505B9E9
:100620003D46002108464FF00000BAF1000F00F4EB
:10063000400005DA00EB80004FF4400101EA500071
:100640004FEA9059B9F1010F00DDB9460A9850EA16
:100650004A000ED044F61050A5F2FF3545432F1442
:10066000B8F1000F1ED07542291E1EDDC9F100022F
:100670001CE0B8F1010F4FF0000001D0302103E081
:10068000F24305E02154401CB042FBDB304600221F
:10069000002121540B99C1F80880C1E900200FB056
:1006A000BDE8F08FBD1B6D1CDEE74A4600DA6942EB
:1006B00006A800F069FA06AB93E8070003AB83E8ED
:1006C000070050460A9900F043FB8DE80700A0F5AB
:1006D00000501F3800900398002D09DD42F21F01E1
:1006E0004A46084403A90390684600F0A2FD08E0CA
:1006F000A0F500504A461F3803A90390684600F051
:10070000ACFD8DE807000004000C03D04FF0FF3073
:10071000410800E01046B8F1000F03D0002200921B
:1007200015461EE0751E05D400F090F93032625572
:100730006D1EF9D5B3460122084302D000227F1C6A
:1007400004E02078302801D100227F1E002A09977A
:1007500086D01DE0112D07DA00F078F930326255AD
:100760006D1C50EA0102F5D1084302D00098C8B1CF
:100770000EE00021681E05E0235C625C6354225495
:10078000401E491C8142F7DBAB46A81B401E099066
:10079000002004F80B000B98099AC0F80880C0E903
:1007A000002B7CE711264FF0000859E72DE9F04FA8
:1007B00088460446D21D22F0070191B0D1E900011C
:1007C000CDE90A0103F030F902460B98C00F01D0C1
:1007D0002D2007E02068810701D52B2002E0202191
:1007E00001EAC000032A099001D0072A05DB03466D
:1007F0004146204600F088F90BE12078800601D5BB
:10080000E06900E00620B8F1650F814606D0B8F136
:10081000660F18D0B8F1670F70D131E00020B9F140
:10082000110F009001DB112301E009F101030AAA75
:1008300001A90CA8FFF7E4FEDDE90C70002609F120
:100840000105834647E001204B4600904FF00047EA
:100850000AAA01A90CA8FFF7D3FEDDE90DB00C9997
:100860005D46002610B909F101000D18B9EB05002D
:1008700003D4C0F1FF3609F10105A5EB09002BE017
:10088000B9F1010F01DA4FF001090020B9F1110FA0
:100890000090484601DD112300E003460AAA01A9A1
:1008A0000CA8FFF7ADFEDDE90C704D46002683462F
:1008B000207800070AD4AB4500DA5D4601A8012D77
:1008C00004DD411911F8011C302907D04F4502DA27
:1008D00017F1040F04DA012082460FE06D1EEEE7E7
:1008E000002F02DCED1B3E4403E0781CA84200DD33
:1008F0007D1CB81B00F1010A4FF00047207800076B
:1009000003D4AA4501DB4FF0FF3A0021B7F1004FB5
:100910000DF143088DF8431024D002202B23002F23
:1009200001DA7F422D230A21021EA0F1010000DC22
:100930005FB197FBF1FC97FBF1F201FB1C7C1746C2
:100940000CF1300C08F801CDEEE7A8F101000370BE
:100950002188090501D5452100E06521A0F10108A4
:1009600000F8011C09980FA9A1EB0807FF1D00B1B1
:100970000120411901EBEA70A1693844081A401EB0
:10098000A0612078C00602D42046AFF30080099809
:1009900028B1D4E901219047206A401C20622078C8
:1009A000C00622D52046AFF300801EE0002E04DBF7
:1009B000B34502DD01A8805D00E03020D4E90121CB
:1009C0009047206A401C2062761CAAF101005FEA71
:1009D000000A0AD100F032F8C0680168405CD4E92E
:1009E00001219047206A401C2062281EA5F10105C4
:1009F000DCDC07E0D4E9012118F8010B9047206AFC
:100A0000401C2062381EA7F10107F3DC2046AFF33B
:100A10000080032011B043E6074B70B50D467B44C0
:100A200000F05FF80446284600F01CF910B14FF0C2
:100A3000FF3070BD204670BD4F3100000048704748
:100A4000B0010020004870479001002030B5B0F19F
:100A50000A024FEA900E71F100034EEA817EB0EB7C
:100A60000E0061EB91014FEA101E4EEA017E10EB81
:100A70000E0041EB11114FEA102E4EEA016E10EB01
:100A80000E0041EB11214FEA104E4EEA014E10EBE1
:100A90000E0041EB1141401841F100014FEAD00036
:100AA00040EA41704FEAD10110EB80054FEA810422
:100AB00044EA907444EB01046D1944EB0404521BA6
:100AC000A3414FF0000348BF0A3200D530BD401C9F
:100AD00041F1000130BD000001694A1C0261087843
:100AE000704700B58FB0CDE901310021059105496E
:100AF0007944CDE9031011466846FFF74FFC0FB06B
:100B000000BD0000E5FFFFFF2DE9F0411F46044650
:100B100003260168072A01F4006004DB08B116A56A
:100B200005E016A503E008B115A500E015A521F024
:100B300010002060A069C01EA0610FB1401EA0611E
:100B40002046AFF300804FB1D4E9012138469047E9
:100B5000206A401C2062C01C206206E0206AFAE77E
:100B6000D4E9012115F8010B9047761EF8D22046F2
:100B7000AFF30080BDE8F0814E414E006E616E0023
:100B8000494E4600696E66002DE9F04781461646DB
:100B90008AB0334878440DC88DE80D003048784459
:100BA000801C03AC0DC884E80D0041F69B3008445E
:100BB000372190FBF1F290FBF1F5A5F1800501FBE7
:100BC00012041B3C02D56442012000E00020DFF843
:100BD00090A080460027FA44AAF1BE0A0DE0E00783
:100BE00009D03246684607EB47010AEB810100F065
:100BF00034FB8DE8070064107F1C002CEFD1184FE8
:100C00007F44AC3F18E0E80714D007EB04100DF167
:100C1000180A90E80E008AE80E00C068F04201D180
:100C200098190890324606A903A800F016FB03ABFA
:100C300083E807006D10641C002DE4D1324669463C
:100C4000B8F1000F03A802D000F0F3FA01E000F0C1
:100C500004FBC9E90001C9F808200AB0BDE8F08723
:100C6000083E0000007B00F080007047004870479D
:100C7000900100207546FFF7F9FFAE460500694672
:100C8000534620F00700854618B020B5FFF7F0FA6C
:100C9000BDE820404FF000064FF000074FF000087D
:100CA0004FF0000B21F00701AC46ACE8C009ACE8FE
:100CB000C009ACE8C009ACE8C0098D46704710B562
:100CC0000446AFF300802046BDE81040FFF7B5BAF8
:100CD0004FF0013C50F8042B51F8043B9A4221D1CB
:100CE000A2EB0C03934313EACC1317D150F8042B57
:100CF00051F8043B9A4215D1A2EB0C03934313EA3B
:100D0000CC130BD150F8042B51F8043B9A4209D173
:100D1000A2EB0C03934313EACC13DBD04FF000009B
:100D2000704700BFD01A01BAB1FA81F101F0180181
:100D300022FA01F0CB40C1F12001DBB2C0B2C01AEF
:100D40002CFA01F3D11A914311EAC311E6D170478D
:100D50005FEA400C08BF91F0000F4FEA8C234FEA86
:100D6000C12243EA51514FEA1C5018BF00F5F04030
:100D70004FEA300018BF41F000415FEA6C5C00F0C0
:100D80002980BCF1FF3F08BF40F080407047130C42
:100D900006BF12044FF0100C4FF0000C130E04BFEE
:100DA00012020CF1080C130F04BF12010CF1040C19
:100DB000930F04BF92000CF1020CD30F04BF52003A
:100DC0000CF1010C11464FF00002A0F11F00A0EB46
:100DD0000C00704711F0004F08BF704731F0004120
:100DE0003FF4D5AF0B0C06BF09044FF0100C4FF0C9
:100DF000000C0B0E04BF09020CF1080C0B0F04BF12
:100E000009010CF1040C8B0F04BF89000CF1020CDA
:100E1000CB0F04BF49000CF1010CCCF12003A0EB77
:100E20000C0022FA03F302FA0CF241EA030100F18A
:100E30000100704720F07F4C80EA030023F07F47D9
:100E4000ACEB070303F57C5300F0004003F1FF0314
:100E50002DE980494FEA154B09B44FEA144325EABE
:100E60000B4E24EA03480FF2042606EB1327490829
:100E70003E785FEA320203FB0667C7F5000707FB0F
:100E800006F64FEA54374FEAD64606F1020607FB4C
:100E9000066CCCF1005C4FEA1C472CEA074C07FBC0
:100EA00006F40CFB06F504EB15464FEA961634BF24
:100EB00000204FF000404FEAD13706FB07FC4FEA15
:100EC0001C4C0CFB0BF7D21B03FB0CF761EB07016F
:100ED0000CFB0EF7B0EB074072EB17420CFB08F768
:100EE00034BFA2EB0742B2EB074261EB17414FEA76
:100EF0000C444FEA910706FB07FC4FEA1C4C0CFB25
:100F00000BF7B0EBC74072EB573203FB0CF734BF63
:100F1000A2EBC742B2EBC74261EB57310CFB0EF7B5
:100F2000B0EBC70072EB57720CFB08F734BFA2EBB3
:100F3000C702B2EBC70261EB5771039F4FEA8161B1
:100F400041EA921104EBCC044FEAD1374FEA8262B6
:100F500006FB07FC42EA90124FEA80604FEA1C4C05
:100F60000CFB0BF7D21B03FB0CF761EB07010CFB2F
:100F70000EF7B0EB074072EB17420CFB08F734BFDB
:100F8000A2EB0742B2EB074261EB17414FEA8C55E7
:100F90004FEA910704EB9C2406FB07FC4FEA1C4C2C
:100FA0000CFB0BF7B0EBC74072EB573203FB0CF7AF
:100FB00034BFA2EBC742B2EBC74261EB57310CFB27
:100FC0000EF7B0EBC70072EB57720CFB08F734BF9B
:100FD000A2EBC702B2EBC70261EB577115EB4C25D0
:100FE0004FEA816141EA92114FEA82624FEAD137BA
:100FF00042EA901206FB07FC44F100044FEA8060CD
:101000004FEA1C4C0CFB0BF7D21B03FB0CF761EBFC
:1010100007010CFB0EF7B0EB074072EB17420CFB1D
:1010200008F734BFA2EB0742B2EB074261EB17416E
:1010300015EB1C154FEA813141EA92414FEA8232A9
:1010400042EA90424FEA80304FEA0C7644F10004C5
:1010500048EA03434EEA0B484FF0000EB2EB080C8F
:1010600071EB030724BF624639464EEB0E0E4FF07C
:10107000000B0018524149414BEB0B0BB2EB080C33
:1010800071EB03077BF1000B24BF624639464EEB40
:101090000E0E4FF0000B0018524149414BEB0B0B69
:1010A000B2EB080C71EB03077BF1000B24BF624627
:1010B00039464EEB0E0E51EA020718BF46F0010604
:1010C00016EB0E7655F1000254F1000103D5BDE890
:1010D0008901BDE80088BDE88901BDE80048B6196E
:1010E000524141EB0101A3F10103704780807F7EF3
:1010F0007D7C7B7A7978777676757473727171708E
:101100006F6E6E6D6C6C6B6A6A696868676666653F
:101110006464636362616160605F5F5E5E5D5D5CCD
:101120005C5B5B5A5A59595858575756565555553E
:101130005454535352525251515050504F4F4F4E9E
:101140004E4D4D4D4C4C4C4B4B4B4A4A4A494949EC
:10115000484848474747474646464545454444442E
:10116000444343434342424242414141002B26D43F
:10117000770021D01CB54FEA370703B44FF01000B9
:101180004FF010014FF000000FBCBDE810400BF114
:10119000010BBBF1010F08BF5FEA170722BF12F175
:1011A000010211F101014FF0004143F1000300F091
:1011B000004043EA00007047F9D35708DAE746EAEF
:1011C000064613F1400F4FEA16461FDD13F1200FBC
:1011D000DFBF16430A46002120335B42C8D0C3F16B
:1011E000200746EA064602FA07F74FEA164646EA9D
:1011F0000706C3F1200722FA03F201FA07F721FAE2
:1012000003F14FF0000342EA0702B1E746EA0206A3
:1012100046EA06464FEA164646EA0106BCBF46EADB
:101220000646360C4FF000034FF000024FF000016D
:101230009EE72DE9C048934630B491E8380007C8CE
:1012400031EA400C48BF34EA430C03D5FFF7F2FD06
:10125000FFF78CFFF0BCBDE800882DE9C04893463D
:1012600030B491E8380007C810F0804F08BF13F081
:10127000804F03D100F005F8FFF778FFF0BCBDE820
:10128000008820F07F4780EA030023F07F4C07EBC3
:101290000C03A3F57C5300F00040A3F1FE0392F091
:1012A000000F00F0B38095F0000F00F077802DE97B
:1012B00001494FEA11404FEA144621EA004800FB79
:1012C00006FC24EA064708FB06F607FB08F800FBC5
:1012D00007F718EB06484CEB164C4FEA124B18EB8D
:1012E00007484FEA15464CEB174022EA0B4E0BFB22
:1012F00006FC25EA06470EFB06F607FB0EFE0BFB77
:1013000007F71EEB064E4CEB164C4FF000061EEB9B
:10131000074E4CEB174B18EB0B0840F1000018EB95
:101320000E0B58EB000840F100008F1A4FF000013F
:101330003CBFC943661B14BFB5EB040C00213CBF86
:10134000C943F61B4FEA17444EEA8E0E27EA0445BE
:101350004FEA1C4704FB07622CEA074C05FB07F722
:101360000CFB05F604FB0CFC16EB074642EB1742A0
:1013700016EB0C4642EB1C421BEB060658EB020236
:10138000414146EA9E0601D5BDE80189B6195241A0
:1013900041EB0101A3F10103BDE801894FEA1445C6
:1013A0004FEA114724EA054621EA074C05FB07F4FA
:1013B00006FB07F70CFB06F105FB0CFC11EB0741E4
:1013C00044EB17444FEA124711EB0C4144EB1C4429
:1013D00022EA074C05FB07F206FB07F70CFB06F6B3
:1013E00005FB0CFC16EB074642EB174216EB0C46CE
:1013F00042EB1C456A1854F1000148BF7047B6190A
:10140000524141EB0101A3F10103704795F0000F38
:1014100037D04FEA11424FEA144721EA024624EA44
:10142000074C02FB07F106FB07F70CFB06F402FB77
:101430000CFC14EB074441EB17414FEA154714EB42
:101440000C4441EB1C4125EA074C02FB07F506FB67
:1014500007F70CFB06F602FB0CFC16EB074645EB08
:10146000174516EB0C4645EB1C42121951F10001D1
:1014700048BF7047B619524141EB0101A3F1010386
:1014800070474FEA14454FEA114724EA054621EA1E
:10149000074C05FB07F106FB07F70CFB06F24FF0C4
:1014A000000605FB0CFC12EB074241EB174112EB67
:1014B0000C4251EB1C4148BF7047921841EB0101AF
:1014C000A3F10103704700BFFEE7000010B5034A17
:1014D0001189506800F038FA10BD00007C0100202E
:1014E0007047000010B504461B481C494860401571
:1014F0000881194808604FF40040488118A0FEF7A1
:1015000041FF16480C3000F041F813481349486079
:1015100000150881154808600420488114A0FEF7D2
:1015200031FF0E480E3000F031F814480B49486086
:10153000001508810D4808600820488110A0FEF7BA
:1015400021FF0648103000F021F8142203492046FC
:10155000FEF794FF10BD0000000002407C01002057
:10156000E9809AE98193310D0A000000000C0240E5
:10157000E9809AE98193320D0A00000000180240C8
:10158000E9809AE98193330D0A00000070B52DEDD2
:10159000028B04469FED1D0A10EE106A02F074FBE8
:1015A000054629461AA0FEF7EDFE05F0FC0078B9C5
:1015B00002F0A2FB00BFFFF789FF0128FBD0204605
:1015C00002F08FFB204601F09DFC10EE106A10E047
:1015D00005F0FC0113A0FEF7D5FEFF20207060701F
:1015E0009FED150A10EE106A02F040FB02F04CFB72
:1015F0000546304603F00CF941EC180B53EC182B60
:101600000EA0FEF7BFFEBDEC028B70BD0000000017
:10161000E69585E99A9CE4BBA3E7A08125640D0AC1
:1016200000000000E99499E8AFAFE4BBA3E7A08114
:1016300025640D0A0000000000C079C474656D7057
:1016400025660D0A0000000070B50446A56D00F087
:101650008FF9064694F83500022808D0802060658E
:1016600000BF002084F8340000BF012070BD206856
:10167000006820F01600216808602068406920F0AA
:10168000800021684861206C08B9A06C28B12068EE
:10169000006820F00800216808602068006820F0D9
:1016A0000100216808600FE000F062F9801B052846
:1016B0000AD92020606500BF002084F8340000BFF4
:1016C000032084F83500D1E72068006800F00100AD
:1016D0000028E9D194F85C103F208840A86000BF42
:1016E000002084F8340000BF012084F83500002079
:1016F000BCE7014691F83500022803D080204865F8
:1017000001207047052081F835000868006820F046
:1017100001000A6810600020F3E7000070B504467D
:1017200000F026F906462546681C10B104480078EA
:10173000054400BF00F01CF9801BA842FAD370BD1D
:1017400014000020F8B502460B46002500240020B6
:101750000021DEE0012606FA01F51E6806EA05040E
:10176000AC4275D11E7906F00306012E04D01E7915
:1017700006F00306022E13D190684F000326BE40E8
:10178000B0434F00DE68BE40304390605068012691
:101790008E40B0431E79C6F300168E403043506031
:1017A0001E7906F00306032E09D0D0684F000326E9
:1017B000BE40B0434F009E68BE403043D0601E79AB
:1017C00006F00306022E13D1CF0802F1200656F8C8
:1017D00027004E07F70E0F26BE40B0434F07FF0EFF
:1017E0001E69BE403043CF0802F1200646F82700AC
:1017F00010684F000326BE40B0431E7906F0030672
:101800004F00BE40304310605E6806F08056B6F16F
:10181000805F7DD100BF00260096404E366846F4BA
:1018200080463E4F3E603E46366806F4804600964F
:1018300000BF00BF3A4E8F0856F827008E07370FBB
:101840000F26BE40B043374EB24202D1002624E0FC
:101850005EE0354EB24201D101261EE0334EB24267
:1018600001D1022619E0324EB24201D1032614E022
:10187000304EB24201D104260FE02F4EB24201D1C8
:1018800005260AE02D4EB24201D1062605E02C4E77
:10189000B24201D1072600E008268F073F0FBE4065
:1018A00030431F4E8F0846F82700264E3068A0436D
:1018B0005E6806F48036B6F5803F00D12043214EA5
:1018C0003060361D3068A0435E6806F40036B6F519
:1018D000003F00D120431B4E361D3060361D30685E
:1018E000A0435E6806F48016B6F5801F00D1204341
:1018F000144E08363060361D3068A0435E6806F42A
:101900000016B6F5001F00D120430E4E0C36306095
:10191000491C1029FFF41EAFF8BD000044380240F6
:101920000838014000000240000402400008024064
:10193000000C024000100240001402400018024057
:10194000001C0240003C0140024613690B400BB1F1
:10195000012000E0002070470AB1816101E00B0422
:101960008361704701480068000C7047002004E064
:1019700001480068704700000C0000200348006820
:101980000349097808440149086070470C000020A9
:101990001400002010B50A48006840F4007008499F
:1019A00008600846006840F480600860032000F08A
:1019B0007FF80F2000F006F800F02AF8002010BD94
:1019C000003C024070B504460E4800784FF47A712E
:1019D000B1FBF0F00C490968B1FBF0F5284601F0C5
:1019E0003AF808B1012070BD102C07D20022214620
:1019F000501E00F01EF80548046001E00120F2E7E7
:101A00000020F0E71400002000000020100000205B
:101A1000704701460846002809DB00F01F03012239
:101A20009A4043099B0003F1E023C3F8002100BF63
:101A300070472DE9F05F80460D461646002702F0FC
:101A40000BF8074639462A46334601F00700C0F135
:101A5000070ABAF1040F02D94FF0040A01E0C0F1FD
:101A6000070AD14600F1040ABAF1070F02D24FF07B
:101A7000000A01E0A0F1030AD4464FF0010A0AFA75
:101A800009FAAAF1010A0AEA020A0AFA0CFA4FF064
:101A9000010B0BFA0CFBABF1010B0BEA030B4AEA4F
:101AA0000B042146404601F0DFFFBDE8F09F000037
:101AB00000BF00F00702064B19684FF6FF031940FC
:101AC000044B0B4343EA0221014B196000BF7047EE
:101AD0000CED00E00000FA0570B504460D460CB9A7
:101AE000012070BD5848006800F00700A84209D2E4
:101AF00055490D700846006800F00700A84201D063
:101B00000120EEE7207800F0020002281DD12078A5
:101B100000F00400042805D14C48006840F4E0506F
:101B20004A490860207800F00800082805D1474895
:101B3000006840F46040454908604448006820F06F
:101B4000F000A168084341490860207800F00100D6
:101B5000A8B36068012807D13C4808380068C0F382
:101B60004040B8B90120BCE76068022802D0606834
:101B7000032807D1354808380068C0F3406048B9E9
:101B80000120AEE7314808380068C0F3400008B9CA
:101B90000120A6E72D48006820F003006168084393
:101BA0002A490860FFF7E4FE064609E0FFF7E0FE79
:101BB000801B41F28831884202D9032091E707E077
:101BC0002248006800F00C006168B0EB810FEDD195
:101BD0001D48006800F00700A84209D91A490D7095
:101BE0000846006800F00700A84201D0012078E70D
:101BF000207800F00400042807D11448006820F47D
:101C0000E050E168084311490860207800F00800BE
:101C1000082808D10D48006820F46040216940EA96
:101C2000C1000A49086000F03FF808490968C1F39B
:101C30000311074A515CC84006490860064800681D
:101C4000FFF7C0FE00204CE7003C0240083802408D
:101C50000A49000800000020100000200148006828
:101C6000704700000000002000B5FFF7F7FF0449AF
:101C70000968C1F38221034A515CC84000BD0000DD
:101C8000083802401A49000800B5FFF7E7FF044989
:101C90000968C1F34231034A515CC84000BD0000ED
:101CA000083802401A4900082DE9F04700240025B1
:101CB0000026A1462548006800F00C0020B1042849
:101CC00005D008283AD105E0DFF8849039E0DFF844
:101CD000849036E01D48001F006800F03F041B4858
:101CE000001F006800F4800078B11A481749091FE6
:101CF0000968C1F38811A0FB017001462246002348
:101D00003846FEF7C8FA05460EE011480F49091F8C
:101D10000968C1F38811A0FB017001462246002327
:101D20003846FEF7B8FA05460848001F0068C0F3B9
:101D30000140401C4600B5FBF6F902E0DFF81090C8
:101D400000BF00BF4846BDE8F087000008380240E9
:101D50000024F40000127A00F8B504460CB9012002
:101D6000F8BD207800F00100002874D0F948006820
:101D700000F00C0004280DD0F648006800F00C00BC
:101D8000082813D1F348001F006800F48000B0F564
:101D9000800F0BD1EF4808380068C0F3404000289E
:101DA00059D06068002856D10120D9E700BF60688B
:101DB000B0F5803F08D1E7480838006840F480302B
:101DC000E449083908601EE06068B0F5A02F0DD125
:101DD000E0480838006840F48020DE49083908608F
:101DE0000846006840F4803008600CE0D9480838A4
:101DF000006820F48030D749083908600846006838
:101E000020F48020086000BF606890B1FFF7B0FD4B
:101E1000054606E0FFF7ACFD401B642801D903200E
:101E20009EE7CC4808380068C0F340400028F1D055
:101E300011E0FFF79DFD054606E0FFF799FD401B09
:101E4000642801D903208BE7C24808380068C0F332
:101E500040400028F1D1207800F0020002285FD134
:101E6000BC48006800F00C0058B1BA48006800F0A7
:101E70000C0008281CD1B748001F006800F480003F
:101E8000B0B9B44808380068C0F3400020B1E06839
:101E9000012801D0012063E7AE480838006820F02F
:101EA000F800216940EAC100AA490839086037E012
:101EB000E06800B30120A8490860FFF759FD054616
:101EC00006E0FFF755FD401B022801D9032047E734
:101ED000A04808380068C0F340000028F1D09D48B1
:101EE0000838006820F0F800216940EAC1009949EB
:101EF0000839086014E0002097490860FFF738FDB2
:101F0000054606E0FFF734FD401B022801D90320F7
:101F100026E7904808380068C0F340000028F1D157
:101F2000207800F0080008282CD16069A8B10120B1
:101F30008A490860FFF71CFD054606E0FFF718FD1B
:101F4000401B022801D903200AE782486C30006850
:101F5000C0F340000028F1D014E000207F49086061
:101F6000FFF706FD054606E0FFF702FD401B0228CD
:101F700001D90320F4E677486C300068C0F34000D4
:101F80000028F1D1207800F00400042870D1002747
:101F900070483830006800F0805090B900BF0020D1
:101FA00000906C483830006840F080506949383102
:101FB00008600846006800F08050009000BF00BF35
:101FC00001276748006800F48070B0B96448006871
:101FD00040F4807062490860FFF7CAFC054606E0DD
:101FE000FFF7C6FC401B022801D90320B8E65C4875
:101FF000006800F480700028F2D000BFA0680128BB
:1020000008D154486830006840F0010051496831F7
:1020100008601DE0A06805280DD14E4868300068B2
:1020200040F004004B49683108600846006840F001
:10203000010008600CE047486830006820F00100AB
:102040004449683108600846006820F004000860D0
:1020500000BFA068A8B1FFF78BFC054609E0FFF7B9
:1020600087FC401B41F28831884202D9032077E681
:1020700026E0384868300068C0F340000028EED001
:1020800013E0FFF775FC054608E0FFF771FC401B05
:1020900041F28831884201D9032061E62D48683039
:1020A0000068C0F340000028EFD1012F07D1294874
:1020B0003830006820F0805026493831086000BF71
:1020C000A069002845D02348006800F00C000828CB
:1020D0005DD0A069022845D100201F490866FFF79E
:1020E00047FC054606E0FFF743FC401B022801D9E8
:1020F000032035E6174808380068C0F34060002820
:10210000F1D1D4E907010843616A40EA8111012253
:10211000A06AC2EB500041EA00412C20005D41EA78
:1021200000600C49091F086001200B490866FFF791
:102130001FFC054606E0FFF71BFC401B022801D9E7
:1021400003200DE6034808380068C0F3406000280B
:10215000F1D049E00838024000004742800E474273
:1021600000700040002021490866FFF701FC054689
:1021700006E0FFF7FDFB401B022801D90320EFE535
:102180001B480068C0F340600028F2D12CE0A06931
:10219000012800D1E4E51648001D0668A069012861
:1021A00020D006F48001E06981421BD106F03F0196
:1021B000206A814216D147F6C0703040616AB0EBA8
:1021C000811F0FD106F440310122A06AC2EB5000FA
:1021D000B1EB004F06D106F070612C20005DB1EB31
:1021E000006F01D00120BBE50020B9E500004742A7
:1021F0000038024010B504460CB9012010BD606AD9
:1022000038B96068B0F5827F00D105E00021E16156
:1022100002E0002121616161A06AB0F5005F00D198
:1022200000BF94F8510028B9002084F850002046DF
:1022300000F050F8022084F851002068006820F077
:10224000400021680860A08800F48270218901F4B0
:1022500004410843A18901F400610843217C01F095
:1022600002010843217D01F001010843218B01F4A3
:1022700000710843217F01F0380108432021095DE6
:1022800001F080010843218D01F4005108432168C9
:1022900008600421A06901EA104094F8241001F0BC
:1022A0001001084321684860A06AB0F5005F03D1BF
:1022B000A08D80B2216808612068C06920F40060A8
:1022C0002168C86100206065012084F85100002069
:1022D00094E7000010B586B00446142101A8FEF76B
:1022E000FFF82349206888423FD100BF00200090BA
:1022F0002048006840F400401E4908600846006815
:1023000000F40040009000BF00BF00BF002000901C
:1023100018481038006840F0040016491039086069
:102320000846006800F00400009000BF00BF00BF36
:10233000002000900846006840F0800008600846D1
:10234000006800F08000009000BF00BF4FF4E05034
:1023500001900220029000200390032004900620A8
:10236000059001A90448FFF7EDF906B010BD000083
:10237000003C004040380240000802402DE9FC4784
:102380000446884617461D46002001908146606835
:10239000B0F5827F0DD1A06858B9042084F85100AF
:1023A0003B46424641462046009500F0EBF9BDE829
:1023B000FC8700BF94F85000012801D10220F6E705
:1023C000012084F8500000BFFFF7D2FA064694F8C7
:1023D0005100012802D04FF00209D6E0B8F1000FF9
:1023E00000D017B94FF00109CFE0042084F8510064
:1023F00000206065C4F83880A787E7872063A0863F
:10240000E08620646064A06AB0F5005F10D100BF70
:102410002068006820F40050216808602068006887
:1024200040F400502168086000BFE08F401EE08744
:10243000A068B0F5004F0BD12068006820F0400084
:10244000216808602068006820F4804021680860E6
:102450002068006800F04000402805D0206800682F
:1024600040F0400021680860E068F8B91AE0206890
:10247000806800F0010050B12068007BA16B0870FB
:10248000A06B401CA063E08F401EE0870AE0FFF7CE
:102490006FFA801BA84201D3681C00B915B94FF030
:1024A000030972E0E08F0028E1D11EE01AE0206805
:1024B000806800F0010050B12068C068A16B0880FE
:1024C000A06B801CA063E08F401EE0870AE0FFF74E
:1024D0004FFA801BA84201D3681C00B915B94FF010
:1024E000030952E0E08F0028E1D1A06AB0F5005F57
:1024F00030D12068006840F48050216808602B4685
:10250000012211462046009600F0E6FE10B14FF081
:1025100003093AE0E068B0F5006F04D12068C068B4
:10252000A16B088003E02068007BA16B08702B463C
:10253000012211462046009600F0CEFE30B1606DBB
:1025400040F0020060654FF003091EE02068C0689B
:10255000019000BF32462946204600F03DFE08B1FA
:10256000202060652068806800F01000102807D1E6
:10257000606D40F0020060654FF6EF702168886082
:10258000606D08B14FF0010900BF012084F85100CF
:1025900000BF002084F8500000BF484607E72DE93F
:1025A000F84F0446884616461D464FF0000A00BF05
:1025B00094F85000012802D10220BDE8F88F0120D4
:1025C00084F8500000BFFFF7D3F90746B14694F8EE
:1025D0005100012802D04FF0020AC9E0B8F1000F03
:1025E00000D016B94FF0010AC2E0032084F8510070
:1025F00000206065C4F83080A686E686A063A087C8
:10260000E08760642064A068B0F5004F0BD12068BB
:10261000006820F04000216808602068006840F4ED
:10262000804021680860A06AB0F5005F0DD100BF4E
:102630002068006820F40050216808602068006865
:1026400040F400502168086000BF2068006800F076
:102650004000402805D02068006840F04000216814
:102660000860E068B0F5006F2FD1606810B1B9F173
:10267000010F09D1206B00882168C860206B801C85
:102680002063E08E401EE0861BE02068806800F03A
:10269000020002280AD1206B00882168C860206BE4
:1026A000801C2063E08E401EE0860AE0FFF760F9A0
:1026B000C01BA84201D3681C00B915B94FF0030A2A
:1026C00056E0E08E0028E0D12EE0606810B1B9F14C
:1026D000010F09D1206B007821680873206B401C22
:1026E0002063E08E401EE0861BE02068806800F0DA
:1026F000020002280AD1206B007821680873206B41
:10270000401C2063E08E401EE0860AE0FFF730F9AF
:10271000C01BA84201D3681C00B915B94FF0030AC9
:1027200026E0E08E0028E0D1A06AB0F5005F05D178
:102730002068006840F48050216808603A462946C5
:10274000204600F093FD08B120206065A06850B9D4
:1027500000BF002000902068C0680090206880685A
:10276000009000BF00BF606D08B14FF0010A00BFCC
:10277000012084F8510000BF002084F8500000BF01
:1027800050461AE72DE9F04F85B004468846914639
:102790001D460E9E00200490012002900020019012
:1027A00000BF94F85000012803D1022005B0BDE815
:1027B000F08F012084F8500000BFFFF7D9F80746DA
:1027C00094F851B060680390AA46BBF1010F0BD09A
:1027D0000398B0F5827F04D1A06810B9BBF1040F53
:1027E00002D0022001902CE1B8F1000F03D0B9F122
:1027F000000F00D015B90120019022E194F851009A
:10280000042802D0052084F8510000206065C4F837
:102810003890E587A587C4F83080E586A5862064D2
:102820006064A06AB0F5005F0DD100BF2068006849
:1028300020F40050216808602068006840F40050CF
:102840002168086000BF2068006800F04000402850
:1028500005D02068006840F0400021680860E0680A
:10286000B0F5006F56D1606810B1BAF1010F09D10F
:10287000206B00882168C860206B801C2063E08E7C
:10288000401EE0863FE02068806800F002000228D9
:102890001CD1E08ED0B10298012817D1206B00889E
:1028A0002168C860206B801C2063E08E401EE0869B
:1028B00000200290E08E48B9A06AB0F5005F05D113
:1028C0002068006840F480502168086020688068B3
:1028D00000F0010068B1E08F58B12068C068A16BBA
:1028E0000880A06B801CA063E08F401EE087012061
:1028F0000290FFF73DF8C01BB04204D3701C10B12A
:10290000032001909DE0E08E0028BCD1E08F0028DC
:10291000B9D156E0606810B1BAF1010F09D1206B4E
:10292000007821680873206B401C2063E08E401EF5
:10293000E08640E02068806800F0020002281CD198
:10294000E08ED0B10298012817D1206B0078216861
:102950000873206B401C2063E08E401EE086002040
:102960000290E08E48B9A06AB0F5005F05D12068FA
:10297000006840F48050216808602068806800F09A
:10298000010068B1E08F58B12068C068A16B087081
:10299000A06B401CA063E08F401EE08701200290E6
:1029A000FEF7E6FFC01BB04201D3701C00B916B998
:1029B0000320019045E0E08E0028BBD1E08F002885
:1029C000B8D1A06AB0F5005F12D13346012211469A
:1029D0002046009700F080FC30B1606D40F00200AE
:1029E0006065032001902CE02068C068049000BF5F
:1029F0002068806800F01000102809D1606D40F058
:102A0000020060654FF6EF70216888600120019038
:102A10003A463146204600F029FC20B101200190C1
:102A2000202060650DE0A06850B900BF0020009034
:102A30002068C068009020688068009000BF00BFD8
:102A400000BF012084F8510000BF002084F850002E
:102A500000BF0198AAE670B504462546681EB0F18D
:102A6000807F01D301200FE0681E4FF0E021486114
:102A70000F214FF0FF3000F0F7FF00204FF0E02172
:102A8000886107200861002070BD704770470146CB
:102A90000022002391F83D2091F83E3042EA0300E5
:102AA000704700002DE9F84F04462068056820684B
:102AB000C668206847694FF00009CA4605F00F094B
:102AC000B9F1000F0AD105F0200038B106F020005E
:102AD00020B1204600F0B5FDBDE8F88FB9F1000F38
:102AE00072D007F0010018B906F4907000286BD07E
:102AF00005F0010030B106F4807018B1206C40F090
:102B00000100206405F0040030B107F0010018B1A5
:102B1000206C40F00200206405F0020030B107F0A4
:102B2000010018B1206C40F00400206405F008009A
:102B300048B106F0200010B907F0010018B1206C70
:102B400040F008002064206C70B305F0200028B12C
:102B500006F0200010B1204600F073FD20684069A7
:102B6000C0F3801A206C00F0080010B9BAF1000F11
:102B700023D0204600F03AFD2068406900F0400074
:102B8000402816D12068406920F040002168486143
:102B9000A06B50B15648A16B0865A06BFEF7A9FD6C
:102BA00010B1A06B016D88470CE02046FFF76EFF67
:102BB00008E02046FFF76AFF04E02046FFF766FFC3
:102BC0000020206488E7FFE7206B012879D105F019
:102BD0001000002875D006F01000002871D000BF4A
:102BE00000200090206800680090206840680090F5
:102BF00000BF00BF2068406900F04000402839D184
:102C0000A06B006840681FFA80F8B8F1000F30D060
:102C1000A08D40452DDDA4F82E80A06BC069B0F5D5
:102C2000807F1FD02068C06820F480702168C86051
:102C30002068406920F001002168486120684069EF
:102C400020F0400021684861202084F83E000020E8
:102C500020632068C06820F010002168C860A06B65
:102C6000FEF7F2FCA08DE28D801A81B22046FFF7BC
:102C70000CFF31E7A08DE18D401A1FFA80F8E08D3E
:102C8000E8B1B8F1000F1AD02068C06820F4907045
:102C90002168C8602068406920F00100216848610F
:102CA000202084F83E00002020632068C06820F0C7
:102CB00010002168C86041462046FFF7E6FE0BE79A
:102CC000FFE705F0800030B106F0800018B1204623
:102CD00000F04FFE00E705F0400030B106F0400084
:102CE00018B1204600F09DFCF6E600BFF4E60000B7
:102CF000D935000810B504460CB9012010BDA069F3
:102D000000B100E000BF94F83D0028B9002084F82D
:102D10003C00204600F028F8242084F83D0020687C
:102D2000C06820F400502168C860204600F0E8FC2C
:102D30002068006920F4904021680861206840699B
:102D400020F02A00216848612068C06840F40050E3
:102D50002168C86000202064202084F83D0084F8A9
:102D60003E000020CAE7000010B586B004462D4999
:102D70002068884254D100BF00BF002000902A483C
:102D8000006840F01000284908600846006800F01C
:102D90001000009000BF00BF00BF00BF00BF0020B8
:102DA000009021481438006840F008001E4914398A
:102DB00008600846006800F00800009000BF00BFEF
:102DC00000BF00BF00BF002000900846006840F030
:102DD000020008600846006800F00200009000BF92
:102DE00000BF00BF4020019002200290012003900C
:102DF000022004900720059001A90C48FEF7A2FCD0
:102E0000802001900720059001A90848FEF79AFC50
:102E10002520FEF7FEFD032211462520FEF709FEC0
:102E200006B010BD001001404438024000040240CA
:102E300070B504460D46164694F83E00202816D17B
:102E400005B10EB9012070BD00BF94F83C00012807
:102E500001D10220F7E7012084F83C0000BF0020E8
:102E6000206332462946204600F060FDEBE7022051
:102E7000E9E700001D4A0168914236D11C490988E2
:102E800001F4004189BB1A49098801F4804171B1FC
:102E9000184909780A2903D00021154A118024E035
:102EA0001349098841F40041114A11801DE011497C
:102EB00009780D2906D10E49098841F480410C4A50
:102EC000118012E00B490978094A1288C2F30D02F9
:102ED000094B995406490988491C054A1180114635
:102EE0000988C72901DD00211180704700100140C9
:102EF000080000200A00002018000020704700BFD2
:102F0000FEE70000F0B52DED108B85B005469FED76
:102F10009E0AF0EE40EA9FED9D0AB0EE40EA9FED7A
:102F20009C0AF0EE409A287804026878044364080A
:102F300000EE104AB8EE400A10EE100A01F068FCEC
:102F400041EC1C0B9FED930B53EC102B01F054F84C
:102F500041EC1B0B9FED910B53EC102B01F0A4F9EE
:102F600041EC1A0B00F06EFF08EE900AB1EE4E0A2B
:102F700010EE106A2EEE0E0AF1EE000A00EEE90ADB
:102F80008DED030AB1EE000A29EE800AC0EE2E0A8A
:102F9000CDED020AB0EE000A29EE800A10EE107A9A
:102FA0009DED030ADDED020A00EEA80AB0EE409A9C
:102FB000384601F02DFC41EC1D0B304601F028FC99
:102FC00041EC1A0B19EE100A01F022FC41EC1C0B2B
:102FD000B0EE4C0AF0EE6C0A00F05AFDB0EE40BACA
:102FE000F0EE60BA53EC1A2B51EC1B0B00F05CFFB7
:102FF00053EC1D2BCDE900019DED000B51EC100BA6
:1030000000F0FAFF41EC1F0B00F01CFF09EE100A64
:10301000B5EEC09AF1EE10FA05DBB0EE490A05B044
:10302000BDEC108BF0BDB0EE688A9FED5E0AB0EE8D
:10303000409A18EE100A01F0EBFB41EC1D0B9FEDDE
:103040005A0B53EC102B01F02FF941EC1B0B19EE2E
:10305000100A01F0DDFB41EC1C0B53EC1B2B00F0C4
:1030600023FF41EC1A0B00F0EDFE09EE100AB0EE62
:10307000688A28EE080AB0EE408A18EE100A01F0BD
:10308000C7FB41EC1C0B9FED4A0B53EC102B01F0DE
:103090000BF941EC1A0B19EE100A01F0B9FB41ECE7
:1030A0001B0B53EC1A2B00F0FFFE41EC1D0B00F044
:1030B000C9FE09EE100A28EE280AB0EE408A18EE82
:1030C000100A01F0A5FB41EC1D0B9FED3B0B53ECEF
:1030D000102B01F0E9F841EC1B0B19EE100A01F07E
:1030E00097FB41EC1C0B53EC1B2B01F0A7FA41ECB6
:1030F0001A0B00F0A7FE09EE100A28EE280AB0EE1F
:10310000408A18EE100A01F083FB41EC1C0B9FED86
:103110002C0B53EC102B01F0C7F841EC1D0B19EEF2
:10312000100A01F075FB41EC1B0B53EC1D2B01F059
:1031300085FA41EC1A0B00F085FE09EE100A28EE24
:10314000280AB0EE408A18EE100A01F061FB41EC4B
:103150001C0B9FED1D0B53EC102B01F0A5F841EC5F
:103160001D0B19EE100A01F053FB41EC1B0B53EC45
:103170001D2B00F099FE41EC1A0B00F063FE09EEE6
:10318000100AB0EE490A4AE700007A443211803B47
:103190007F051BB5000000000000E04000000000BB
:1031A00000CCB0401F0572C3F163CC5D4BC8014039
:1031B000BB82C87D062F653F93C266C7E03DD43E03
:1031C000CE563151E2425E3E3EFAE46127F3E43DE1
:1031D00000BFFEE770477047F8B504460E46154637
:1031E0006068B0F5827F0DD1A068B0F5004F03D0C4
:1031F000A068B0F5806F05D12068006820F040001D
:10320000216808606068B0F5827F1FD1A068B0F5C2
:10321000806F0DD03346002280212046009500F0BB
:103220005BF808B3606D40F0200060650320F8BDD6
:103230003346002201212046009500F04DF898B158
:10324000606D40F0200060650320F0E73346002207
:1032500001212046009500F03FF828B1606D40F054
:10326000200060650320E2E70020E0E77CB504462B
:103270000D461646164800681821B0FBF1F01549B6
:10328000B0FBF1F04FF47A71484301906068B0F5FB
:10329000827F0DD12B46002280212046009600F02F
:1032A0001BF898B1606D40F02000606503207CBD84
:1032B00000BF019800B908E00198401E0190206805
:1032C0008068C0F3C0100028F3D100BF0020EEE7F3
:1032D0000000002040420F002DE9F84F04460D4643
:1032E00090461E46DDF82890FEF742FBA0EB090051
:1032F000371AFEF73DFB82462C480068C0F3CB30FE
:103300007843009045E0701C002842D0FEF730FB67
:10331000A0EB0A00B84200D2A7BB2068406820F0AA
:10332000E000216848606068B0F5827F0DD1A06838
:10333000B0F5004F03D0A068B0F5806F05D12068CC
:10334000006820F0400021680860A06AB0F5005FC6
:103350000DD100BF2068006820F40050216808608B
:103360002068006840F400502168086000BF012018
:1033700084F8510000BF002084F8500000BF0320F3
:10338000BDE8F88FFFE7009800B900270098401EBD
:103390000090206880682840A84201D1012000E008
:1033A00000204045AFD10020EAE7000000000020E7
:1033B000704710B5FEF7E2FA10BD00000348006840
:1033C00040F47000014908607047000088ED00E09B
:1033D00000B587B0142102A8FDF782F800BF0020D5
:1033E00001902548006840F008002349086008461D
:1033F000006800F00800019000BF00BF00BF00207F
:1034000001900846006840F04000086008460068E7
:1034100000F04000019000BF00BF00BF00200190FD
:103420000846006840F0010008600846006800F0A7
:103430000100019000BF00BF4815029000200390DA
:10344000049002A90D48FEF77DF94FF480600290C8
:1034500000200390049002A90848FEF773F94FF486
:103460008060029000200390049002A90448FEF7B7
:1034700069F907B000BD000030380240000002408A
:103480000018024008B500BF0020009017480068EF
:1034900040F40040154908600846006800F4004008
:1034A000009000BF00BF1248124908604FF48270BC
:1034B000486000210F488160C16002210161012143
:1034C0004161490281613021C16100210162416293
:1034D00081620A21C162FEF78DFE0648006800681D
:1034E00040F0400003490968086008BD40380240C8
:1034F000003C00402401002000B587B0142102A840
:10350000FCF7EEFF00BF002001903048006840F05B
:1035100004002E4908600846006800F0040001908D
:1035200000BF00BF00BF002001900846006840F0C7
:10353000010008600846006800F00100019000BF2B
:1035400000BF00BF002001900846006840F008005E
:1035500008600846006800F00800019000BF00BF46
:10356000012208211A48FEF7F7F901220421184820
:10357000FEF7F2F90122D1031648FEF7EDF94FF4F8
:103580000040029001200390002004900320059049
:1035900002A91048FEF7D6F80420029001200390FB
:1035A000002004900320059002A90948FEF7CAF8FC
:1035B0000820029001200390002004900320059031
:1035C00002A90348FEF7BEF807B000BD303802403C
:1035D000000C02400000024070B50546AC6B0020B4
:1035E000E085E0842046FFF751FA70BD0168C968A4
:1035F00021F490710268D1600168496921F00101EC
:1036000002685161016B012905D10168C96821F087
:1036100010010268D160202180F83E100021016372
:10362000704710B504462068C06820F0400021684B
:10363000C860202084F83D002046FFF75FFC002092
:1036400010BD70B5044694F83E00222856D1A068FB
:10365000B0F5805F0CD1206950B90025A66A2068BA
:103660004068C0F308003080A06A801CA06215E0AA
:10367000A56A0026A068B0F5805F03D0A06828B9CD
:10368000206918B920684068287004E02068406804
:1036900000F07F002870A06A401CA062E08D401EF0
:1036A00080B2E08540BB2068C06820F0200021681F
:1036B000C8602068C06820F480702168C8602068F5
:1036C000406920F0010021684861202084F83E0014
:1036D000206B01280AD12068C06820F01000216802
:1036E000C860A18D2046FFF7D0F902E02046FFF721
:1036F000C1FB0020206370BD0020FCE70220FAE738
:103700002DE9F84F04462068006920F44050E16834
:103710000843216808612169A0680843616908437A
:10372000E169084300902068C06849F20C61884351
:10373000009908432168C8602068406920F44070FF
:10374000A16908432168486176492068884203D00E
:1037500075492068884203D1FEF796FA814602E057
:10376000FEF782FA8146E069B0F5004F6CD1022085
:103770006168A0FB015003461920A9FB00700146B7
:103780002A463846FCF787FD6421B0FBF1F04FEA8A
:10379000001A02206168A0FB01510B461920A9FB09
:1037A00000712A463846FCF776FD834602206168A0
:1037B000A0FB015003461920A9FB00712A46384698
:1037C000FCF769FD6421B0FBF1F000EBC00101EBF7
:1037D0000010ABEB8000322101EBC0006421B0FB94
:1037E000F1F000F0F8000AEB400A02206168A0FB4B
:1037F000015003461920A9FB007001462A463846AD
:10380000FCF749FD834602206168A0FB0150034696
:103810001920A9FB00712A463846FCF73CFD6421BB
:10382000B0FBF1F000EBC00101EB0010ABEB80004E
:10383000322101EBC0006421B0FBF1F000F0070081
:103840005044216888606AE004206168A0FB015050
:1038500003461920A9FB007001462A463846FCF7AA
:103860001AFD824604206168A0FB0150034619201E
:10387000A9FB007001462A463846FCF70CFD64217E
:10388000B0FBF1F000EBC00101EB0010AAEB8000EF
:10389000322101EB00106421B0FBF1F000F0F00ADE
:1038A00004206168A0FB017003461920A9FB0051A8
:1038B0003A462846FCF7EFFC6421B0FBF1F00AEB36
:1038C000001A04206168A0FB01510B461920A9FBD6
:1038D00000712A463846FCF7DEFC83460420616806
:1038E000A0FB015003461920A9FB007001462A469F
:1038F0003846FCF7D0FC6421B0FBF1F000EBC001CE
:1039000001EB0010ABEB8000322101EB00106421D1
:10391000B0FBF1F000F00F00504421688860BDE872
:10392000F88F0000001001400014014010B503465C
:1039300099629A85DA8500201864222083F83E0077
:1039400000BF002083F83C0000BF1868C06840F446
:1039500080701C68E0601868406940F001001C68D5
:1039600060611868C06840F020001C68E0600020BA
:1039700010BD014691F83D00212828D18868B0F596
:10398000805F0BD1086948B90A6A1088C0F3080043
:103990000B685860086A801C086205E00B6A581CB6
:1039A000086218780B685860C88C401E80B2C884C2
:1039B00058B90868C06820F080000B68D8600868B3
:1039C000C06840F040000B68D860002070470220BB
:1039D000FCE7000070B500240F4D1048FFF762F8B7
:1039E00000BF03E0641CAC4200D904E00B48FFF7C1
:1039F0004EF82028F6D100BF002403E0641CAC423E
:103A000000D906E0012206490448FFF711FA002810
:103A1000F4D100BF70BD0000FFFF0100E0000020F6
:103A20000A00002000BFFEE703B40198410000989F
:103A300050EAC12018BF04204A0D18BF40F0010011
:103A400040F2FF72B2EB515F08BF40F00200012864
:103A500008BF052002B0704702480068C0F302208A
:103A6000704700000CED00E010B5002804DB0A07E9
:103A7000130E054A135406E00A07140E034A00F019
:103A80000F031B1FD45410BD00E400E018ED00E04C
:103A900000B52DED048BB0EE409AF0EE609A83B045
:103AA00051EC190B00F0FEFC41EC180B18EE100A5B
:103AB00018EE901A8DED008B002818BF01200843E6
:103AC00020F00040C0F17F6000F1E040C00F14D052
:103AD00019EE101A19EE900A8DED009B002918BFFF
:103AE0000121084320F00040C0F17F6000F1E04078
:103AF000C00F04BF0120FCF723FDB0EE480A03B05D
:103B0000F0EE680ABDEC048B00BD00BF70470000FA
:103B100011B526E0009CB4F5617F02D94FF46174C1
:103B200000E0009C23464FF0E024A069A82404FB99
:103B30001301002908DB00BF4FF0E024A269824294
:103B40000CDA8A42F8DA09E0084C214400BF4FF051
:103B5000E024A2698242FADD8A42F8DC009CE41A81
:103B60000094009C002CD5D118BD000040900200AC
:103B700000BF054A126802F04002002AF9D0C2B222
:103B8000014B5A60704700000010014086B0FDF7FD
:103B900001FF0723022208214FF4A87000F0B2F8B9
:103BA0004FF4E13000F01CF9FFF76CFCFFF7A4FCC8
:103BB000FFF70EFC08A0FCF7E5FB0BE04FF47A7072
:103BC000FDF7ACFD01A8FDF78DFC4FF47A70FDF711
:103BD000A5FD00BFF2E700000D0AE5BC80E5A78B5C
:103BE000E6B58BE9878F3A0D0A00000001B582B077
:103BF0000D4A518910680022FDF7AEFE3C230122D8
:103C000002A90A48FEF7CBFC3C23012201A9074880
:103C1000FEF7B4FB044A518910680122FDF79CFEAF
:103C20009DF804000EBD00007C010020240100204E
:103C300038B504460D468DF800408DF80150094A0C
:103C4000518910680022FDF787FE3C230222694655
:103C50000548FEF7A4FC034A518910680122FDF7CC
:103C60007BFE38BD7C0100202401002010B500201F
:103C7000FFF7BCFF044604F0D30444F002042146DD
:103C80008020FFF7D5FF10BD70B50020FFF7AEFF15
:103C9000044644F0800404F0F30421468020FFF73A
:103CA000C7FFC820FFF734FF44F088042146802076
:103CB000FFF7BEFFC820FFF72BFF44F08C0421461E
:103CC0008020FFF7B5FF00BF0020FFF78FFF00F057
:103CD0000C000028F8D10720FFF788FF054628468A
:103CE00070BD10B504460120FFF780FF2070022050
:103CF000FFF77CFF607010BD10B5C1218020FFF779
:103D000097FF10BD2DE9F04192B080460C46154654
:103D10001E460027302106A8FCF7E2FB142101A86B
:103D2000FCF7DEFB00BF002000902A48006840F04E
:103D30008050284908600846006800F080500090D4
:103D400000BF00BF00BF002000902348006840F47F
:103D50008040214908600846006800F480400090D7
:103D600000BF00BF012006900004079002200C90C5
:103D700041050D91CDF83C800E941095119606A842
:103D8000FDF7EAFF07461FB1012012B0BDE8F08140
:103D90000F20019002200290002003904FF4A050C9
:103DA00004904FF480500590052101A8FDF794FE82
:103DB00007460FB10120E8E7FDF7D4FD41F201010C
:103DC000884205D10548006840F4807003490860C6
:103DD0000020DAE74038024000700040003C02401A
:103DE00010B5044609480A490860084644600021A5
:103DF0008160C160016181610C214161FEF77AFF40
:103E0000012204490248FFF713F810BD00100140D9
:103E1000E00000200A00002010B500290AD0087830
:103E2000002807D005487844FCF752FF002801D04D
:103E3000002010BD0248784410BD0000B20B000005
:103E4000AA0B000021F00042A2F16052B2F5801FDF
:103E500001F0004328BFD2F17F6C0BD95FEA001C50
:103E600043EAC20242EB507018BF704728BF20F0EF
:103E700001007047B2F5801FBCBF184670474FEA7B
:103E8000410C1CF5001F02D2084600F037BD70B58A
:103E900000F0B4FA00000089FFF7F6BF4FF00040D1
:103EA000A0F580007047000010B591EA030F48BFED
:103EB00083F0004300F1CA83841A71EB030C05D22E
:103EC000121943EB0C03001B61EB0C01DFF824E13A
:103ED0004FEA1154A4EB135C1EEA430F18BF9EEA8D
:103EE000445F73D023EA0E03DCF1200E21EA045173
:103EF00043F4801332D322FA0CFE10EB0E0023FAA7
:103F00000CFE41EB0E01CCF1200E03FA0EFE10EB7D
:103F10000E0051F10001B1F5801FCCF1200E32D21C
:103F200001EB045112FA0EF2BDE8104058BF704781
:103F3000401C38BF5FEA420218BF7047002814BF18
:103F400020F0010041F100014FEA410313F5001F89
:103F500038BF7047A1F1C04100F09EBA012A43EB7F
:103F60000302ACF1200CDCF11F0E32BF4FF0000E4B
:103F700023FA0CF310EB030041EB0451B4EB115F97
:103F8000D0D0A1EB045101F5801149085FEA30005F
:103F900001EB04510ED350F1000038BF12FA0EFEAF
:103FA00008D1BDE81040C9E7401C38BF5FEA4202B3
:103FB000CAD1C3E7BDE810404FEA410313F5001F23
:103FC00038BF7047A1F1C04100F066BA9EEA445F75
:103FD00008D011EA5E0FBDE8104004BF01F00041B7
:103FE00000207047BDE8104070B500F007FA00BF30
:103FF00064FBBE3E0000E0FF2DE9C04130B4DFF8B5
:10400000A0C23CEA111418BF3CEA131400F0EC8083
:1040100081EA03051CEA111444EAD57418BF1CEAAE
:10402000131500F0C780A4EB05044FF0004545EAE6
:10403000C12145EAC32341EA505143EA525304F1F6
:104040007F74994204F500344FEAC0204FEAC2223F
:1040500008BF904200F09C804FEA13650FF24016B3
:10406000765D4FEA134506FB05F7C7F1807706FB3F
:1040700007F74FEAD737A7FB03687642C8F58038C1
:10408000A7FB06CE38BFA8F1010807FB08E64FF0F2
:10409000000EA6FB028CE6FB03CEDCF1000CCEF199
:1040A000004E38BFAEF1010EA6FB0C584FF00007D2
:1040B0004FF00005E6FB0E87A1FB08C6A0FB07CE6C
:1040C00016EB0E0645F10005E1FB076515F1E04E24
:1040D0007EBFA4F580345FEA46066D4116F1800785
:1040E00045F100054FEA17274FEA066647EA0567DC
:1040F000A6F1DE46B6F1805F4FEA15251FD9384696
:1041000024F0010C05EBC471BCF1FE6F01EB0C1146
:1041100002D8F0BCBDE8008124425CBF01F5801EDE
:104120009EEAC47F02D4F0BCBDE80081244238D4AA
:10413000F0BCA1F1C041BDE8004100F0ADB94FEACB
:10414000D22242EA43524FEAD323A7FB02864FEA28
:10415000D02040EA415007FB03661EEA0E0F4FEAEB
:10416000D12105FB026658BFA6EB0056B6EB005600
:104170004FEA520E4EEAC37E18EB0E0E56EB530E6C
:10418000BDD518EB02085E417F1C55F10005B6E76E
:104190004FF480154FF000074FF000064FF0000875
:1041A000ADE7F0BC4FF0000001F1C04101F000416B
:1041B000BDE8008111EA0C1F0CEA131500D00CE0D9
:1041C00013EA0C1F00F025804FF00000F0BC81EADC
:1041D000030101F00041BDE80081F0BCBDE80041F1
:1041E00081EA030100F058B9F0BCBDE8004170B5A8
:1041F00000F004F9097EFC3E00F007B881EA0301F3
:104200004FF0000001F00041704781EA030100F027
:1042100043B9F0BCBDE800414FF0000021497047B0
:10422000FFFDFBF9F7F5F4F2F0EEEDEBE9E8E6E47B
:10423000E3E1E0DEDDDBDAD8D7D5D4D3D1D0CFCD02
:10424000CCCBCAC8C7C6C5C4C2C1C0BFBEBDBCBB3B
:10425000BAB9B8B7B6B5B4B3B2B1B0AFAEADACAB36
:10426000AAA9A8A8A7A6A5A4A3A3A2A1A09F9F9E10
:104270009D9C9C9B9A9999989797969595949393C2
:10428000929191908F8F8E8E8D8C8C8B8B8A898959
:1042900088888787868585848483838282818180DC
:1042A0000000FF070000F87FDFF848C170B51CEA86
:1042B000111E1EBF1CEA13159EEA0C0F95EA0C0F87
:1042C00000F06F8081EA030423EA4C134EEAD47EA7
:1042D00021EA4C1141F4801143F48013AE44A1FB58
:1042E000024CA0FB0365AEF17F7E361955EB0C0541
:1042F000A1FB034C4CF10003A0FB021C16EB0C06C7
:10430000654153F10003094218BF46F0010613F45A
:10431000007F0BD14FEA03314FEA0530340341EA05
:10432000155140EA16506FF003020AE04FEAC3212C
:104330004FEAC520F40241EA555140EA56506FF069
:10434000020202EB2E4201EB025585EACE710AD041
:104350005FEA440C18BF24F0004450F1000041F122
:10436000000120EAD47040F2FE7C624500D270BDAC
:10437000A84214BF4FF080444FF04044002E08BFC5
:104380000024BEF1806FA8BFA1F1C041BDE870401C
:1043900080F282804FF0000001F1C04101F0004145
:1043A00070479EEA0C0F0CEA131518BF95EA0C0F24
:1043B00006D04FF0000081EA030E0EF0004170BD00
:1043C00000F01CF88900013E00F007B800F009B8C1
:1043D0004FEA430C5FEA5C5C08D081EA030100F01D
:1043E0005BB84FEA410C5FEA5C5CF6D14FF000002D
:1043F000014970470000FF070000F87F0EF1020E30
:104400002EF0030E5EF8046B364205D4012A43EB0E
:10441000030515F5001F12D8012841EB010C1CF50E
:10442000001F0CD80ED14FEAD17C15F5001F0CEB04
:104430004C0C0CF1020C08BF4CEBD37C04E04FF0A9
:10444000080C01E04FEAD37C0CEB4C0526FA05F68C
:1044500006F00706B6F1040C06D20EEB860CBDE89A
:1044600070404CF0010C6047DFE80CF0090B0202D1
:104470004FF000414FF00000A1F5002170BD19463A
:104480001046012851EB010418BFD4F5001484BF75
:10449000002001F0004170BD0808A0F500114FEAAE
:1044A000310170472DE9F04101F5801CBCF5001F7A
:1044B000C0F2A9804FEA115C21EA0C510CF1FD0C0D
:1044C00041F480115FEA5C0C0CF5C07C01D3400024
:1044D000494130A4890241EA905187028E0E0A0CAC
:1044E000A45D04FB04F602FB06F6C6F14046A4FBFD
:1044F0000662F60D46EA422606FB06F4A4FB0123FB
:104500005242C3F1404338BF5B1EA6FB0242002467
:10451000E6FB0324D20B42EA4446A6FB0623A1FB9A
:1045200002E2A3FB07E4E3FB61426442C2F1404EB6
:1045300038BFAEF1010EA6FB04234FF00002E6FBEC
:104540000E32A2FB03463400E2FB6264A1FB06E6E6
:10455000A4FB07E8E4FB61687642C8F1405838BF25
:10456000A8F10108A2FB06E4A3FB08E5E2FB6854FE
:10457000A1FB05E6A7FB04E8E1FB648618F1200532
:1045800056F10006A809A8F11B08B10908F03F0878
:10459000B8F10A0F40EA86601CD901EB0C51BDE866
:1045A000F08100BFFCF5EEE8E2DDD8D3CFCBC7C386
:1045B000C0BDB9B6B4B1AEACA9A7A5A3A19F9D9B40
:1045C0009A9896959392908F8D8C8B898887868503
:1045D00084838281A0FB006800FB01F208EB4208A3
:1045E000B8EB872807D5341858EB0104D5D5401C03
:1045F00051F10001D1E7341A78EB0104CDD4401E0B
:1046000071F10001C9E75FEA4C0C5FEA9C5C0DD1D7
:1046100005D34FF0000001F00041BDE8F081BDE896
:10462000F04170B5FFF7EAFE6DDBFFBEBDE8F0417B
:104630004FF00000004970470000F87F10B591EA84
:10464000030F48BF83F000433FF536AC841A71EB8B
:10465000030C07D212198CF0004C43EB0C03001B27
:1046600061EB0C01DFF8A4E14FEA1154A4EB135CF9
:104670001EEA430F18BF9EEA445F00F0B08023EAB1
:104680006E03524221EA0451C3EB6E0338BF5B1E36
:10469000DCF1200E25D322FA0CFE10EB0E0043FABB
:1046A0000CFE41EB0E01CCF1200E03FA0EFE10EBD6
:1046B0000E0051F10001CCF1200E29D412FA0EF2B5
:1046C00001EB0451BDE8104058BF7047401C1CBFAF
:1046D000B2F1004F704700280CBF491C20F00100C8
:1046E000704712EB020E43EB030218BF4FF0010EAE
:1046F0004EEA4202ACF1200CDCF11E0E54D943FA12
:104700000CFE10EB0E0051F1FF31CCF11E0ED5D591
:104710000EF1010E12FA0EFE404141EB010101EBD8
:10472000445C5FEA5C5C10D910EBDE7001EB045175
:1047300038BFBEF1004FBDE8104018BF70470028D9
:104740000CBF491C20F00100704730D24FEAD42C36
:1047500011F5001124F400641BD0B1FA81F20B3A78
:10476000A41AA41ED2F12003914030FA03F3194396
:10477000904001EBCC71002C01EB0451BDE81040DE
:10478000A8BF704701F1C0414FF0000001F00041A7
:104790007047B0FA80F310FA03F100D110BDE41AAB
:1047A000173C4805C90AE4E701EB045110BD491064
:1047B00001EB0451BDE810404FEA300002E04FF039
:1047C000000170474A0008BF0042F8D0B2F5001F50
:1047D00028BF704701F000414FF0000070479EEA8B
:1047E000445F07D011EA5E0FBDE8104004BF00210E
:1047F00000207047BDE8104070B5FFF7FFFD00BF17
:1048000040DFF63E83F00041104670470000E0FFB5
:1048100043004FEAD30C4FEA3C0C43401FBF400714
:104820000CF1605113F0FE4F70471CF0006F03D184
:1048300000200CF0004170470CF0004343EA507038
:1048400010B540EACC0000F00EF800BF0000009266
:104850004FEA0001FFF720BE4FF000414FF000008B
:10486000A1F5002170470EF1020E2EF0030E5EF846
:10487000044B244204D44FEA4102B2F17F4F11D8D5
:104880004FEA4003B3F17F4F0CD80ED14FEAD07CF2
:10489000B2F17F4F0CEB4C0C0CF1020C08BF4CEB4F
:1048A000D17C04E04FF0080C01E04FEAD17C0CEB26
:1048B0004C0324FA03F404F00704B4F1040C06D208
:1048C0000EEB840CBDE810404CF0010C6047DFE8B3
:1048D0000CF0070802024FF00040A0F5800010BD68
:1048E0000846420018BFD2F1807288BF00F0004035
:1048F00010BD4FF04070E1EE100A7047FF2141EA11
:10490000D050C0057047FBF751BF00000000000009
:10491000000001020304060708090000000001026C
:104920000304000002400000000000A0000000009E
:1049300005400000000000C8000000000C4000001E
:104940000000409C00000000194000000020BCBE98
:104950000000000034400000BFC91B8E00000004AE
:10496000B5400000504BCFD06607E2CF01000000F9
:104970006C4100003E8251AADFEEA7340100000026
:10498000D9420000DCB5A0E23A301F97FFFFFFFFDD
:10499000B4450000FD25A0C8E9A3C14FFFFFFFFFFC
:1049A000FF3F00000000008000000000FF3F00000B
:1049B0000000008000000000F44900080000002012
:1049C00018000000C40100080C4A0008180000206C
:1049D000D8050000E00100081C00000043000000B2
:1049E000F8FFFFFF0C0000000E0000000F000000A9
:1049F0002E0000000024F400000000000000000071
:0C4A000000000000100000000100000099
:040000050800018965
:00000001FF
